:10000000FDC0000007C1000005C1000003C10000E1
:1000100001C10000FFC00000FDC00000FBC00000E7
:10002000F9C00000F7C00000F5C00000F3C00000F8
:10003000F1C00000EFC00000EDC00000EBC0000008
:10004000E9C00000E7C00000E5C00000E3C0000018
:10005000E1C00000DFC00000DDC00000DBC0000028
:10006000D9C00000D7C00000D5C00000D3C0000038
:10007000D1C00000CFC00000CDC00000CBC0000048
:10008000C9C00000C7C00000C5C00000C3C0000058
:10009000C1C00000BFC00000BDC00000BBC0000068
:1000A000B9C00000B7C00000B5C00000B3C0000078
:1000B000B1C00000AFC00000ADC00000ABC0000088
:1000C000A9C00000A7C00000A5C00000A3C0000098
:1000D000A1C000009FC000009DC000009BC00000A8
:1000E00099C0000097C0000095C0000093C00000B8
:1000F00091C000008FC000008DC000008BC00000C8
:1001000089C0000087C0000085C0000083C00000D7
:1001100081C000007FC000007DC000007BC00000E7
:1001200079C0000077C0000075C0000073C00000F7
:1001300071C000006FC000006DC000006BC0000007
:1001400069C0000067C0000065C0000063C0000017
:1001500061C000005FC000005DC000005BC0000027
:1001600059C0000057C0000055C0000053C0000037
:1001700051C000004FC000004DC000004BC0000047
:1001800049C0000047C0000045C0000043C0000057
:1001900041C000003FC000003DC000003BC0000067
:1001A00039C0000037C0000035C0000033C0000077
:1001B00031C000002FC000002DC000002BC0000087
:1001C00029C0000027C0000025C0000023C0000097
:1001D00021C000001FC000001DC000001BC00000A7
:1001E00019C0000017C0000015C0000013C00000B7
:1001F00011C000000FC000000DC0000011241FBE80
:10020000CFEFDFE3DEBFCDBF00E00CBF0E941814CC
:100210000C94C814F5CEFC0180E090E280839183B9
:100220009170DB018D939C938181869580831182EF
:1002300008950F931F9340E358E060E070E08091D1
:10024000D10080FDFCCF82EE8093D000000082E2DE
:100250008093D0008AE38093CA014093C001BB27FA
:10026000A72F962F852F8093C1011092C20180E0A5
:1002700090E2AA2797FDA095BA2F0197A109B1098D
:10028000840F951FA61FB71F8093C401492F5A2FB3
:100290006B2F77274093C501CD01AA27BB278093F9
:1002A000C60188ED84BF8091CB0181608093CB0132
:1002B0008091CF0187FDFCCF8091D10080FDFCCFE4
:1002C0004091D7000091D6008091D5009091D40044
:1002D00010E020E030E0980111270027342B092B93
:1002E0001092D000182BB801C9011F910F910895E9
:1002F000AF92BF92CF92DF92EF92FF920F931F9334
:10030000CF93DF9300D01F92CDB7DEB78C016A0187
:100310007B018FEF9FEFF80180839183BE016F5FB8
:100320007F4FCE01039677DF8B819C81A0E0B0E008
:10033000C816D906EA06FB0618F480E092E007C06A
:10034000C816D906EA06FB0629F489819A818B83AF
:100350009C8302C01B821C8289E0CC0CDD1CEE1C3D
:10036000FF1C8A95D1F780E398E0C80ED91EE11CE6
:10037000F11C58010BC0C701B601620F731F811D2C
:10038000911D40E065D0F50181935F019501201B2F
:10039000310B8B819C812817390768F3C90124969A
:1003A000CDBFDEBFDF91CF911F910F91FF90EF90F6
:1003B000DF90CF90BF90AF9008952FEF31E0FC0118
:1003C000E20FF31F5081FB01E20FF31F408154172E
:1003D00029F0451748F421E030E008C021503109E8
:1003E00070F720E030E002C02FEF3FEFC901089521
:1003F000BF92CF92DF921F93CF93DF93DC01CB01AB
:10040000142FE9013FB7F894E0E0FFE00F921F924C
:100410007DEF6FEF5FEF40E8D92EC82EBA2E209106
:100420003C002F9321E020933C00212F1D2E0C2E09
:1004300019950F9000923C001F900F902F3FF9F3F9
:100440003FBFDF91CF911F91DF90CF90BF90089574
:10045000CF92DF92EF92FF921F936C01EE24FF2464
:10046000FB0110913B00C0923B004093CA01D8951C
:10047000802D10933B001F91FF90EF90DF90CF9065
:1004800008958F929F92AF92BF92CF92DF92EF9298
:10049000FF920F931F93CF93DF931F92CDB7DEB7D9
:1004A0004A015B0139E0880C991CAA1CBB1C3A95D7
:1004B000D1F78C01C12CD12C7601C701B601680D92
:1004C000791D8A1D9B1D422F2983C2DFF80181936C
:1004D0008F01FFEFCF1ADF0AEF0AFF0A2981C1144B
:1004E00082E0D806E104F10441F780E092E00F9049
:1004F000DF91CF911F910F91FF90EF90DF90CF9000
:10050000BF90AF909F908F900895AF92BF92CF927F
:10051000DF92EF92FF920F931F93CF93DF931F927F
:10052000CDB7DEB75C016A017B0149E0CC0CDD1C74
:10053000EE1CFF1C4A95D1F700E012E001501109B2
:10054000C701B601600F711F811D911D422F2983C4
:100550007FDFF501E00FF11F90812981981729F0C5
:10056000981748F42FEF3FEF08C00115110531F738
:1005700020E030E002C021E030E0C9010F90DF91BF
:10058000CF911F910F91FF90EF90DF90CF90BF9090
:10059000AF90089520E075CF20E0B7CFE8E0FFE00E
:1005A0007DEF6FEF5FEF40E820913C002F9321E05B
:1005B00020933C0019950F9000923C00822F80956B
:1005C0000895EAE0FFE020913C002F9321E0209382
:1005D0003C0019950F9000923C002F3F19F4BB2767
:1005E000A0E207C0203019F4BFEFAFEF02C0BB2775
:1005F000A22FCD010895EEE0FFE020913C002F9363
:1006000021E020933C00282F19950F9000923C0088
:10061000822F08952F923F924F925F926F927F9216
:100620008F929F92AF92BF92CF92DF92EF92FF9202
:100630000F931F93CF93DF93EC014B0169017A0174
:1006400059E0CC0CDD1CEE1CFF1C5A95D1F716E2CC
:100650001093CA012091CB01216018ED1093340052
:100660002093CB011091CF011078E1F716012701FB
:10067000612C712CF401E60DF71DB180A12C808155
:100680009501282B10913C008A818F778CBFE881DF
:10069000F98143E2C201B101199510933C0082E057
:1006A000680E711C82E0280E311C411C511C611423
:1006B00082E07806F9F610913C008A818F778CBF32
:1006C000E881F98120E030E0402FC701B60119959B
:1006D00010933C0080E092E0DF91CF911F910F9149
:1006E000FF90EF90DF90CF90BF90AF909F908F9052
:1006F0007F906F905F904F903F902F9008958F92D2
:100700009F92AF92BF92CF92DF92EF920F93CF93CF
:10071000DF936C01EB0149015A01202FB501A401BF
:10072000CE01F3DE892B41F00E2DA5019401BE010F
:10073000C60170DF9C0102C020E032E0C901DF91F8
:10074000CF910F91EF90DF90CF90BF90AF909F909F
:100750008F900895EF92FF920F931F93CF93DF93A3
:10076000CDB7DEB72797CDBFDEBF7C019A01AB01C5
:1007700008EF11E0B80180E82C833D834E835F834E
:1007800041D009831A838B830FE22C813D814E81F6
:100790005F81B701CE0101963DDF2796CDBFDEBF59
:1007A000DF91CF911F910F91FF90EF900895CF921D
:1007B000DF92EF92FF92CF93DF93EC016A017B010E
:1007C000EBDE892B51F0B701A601CE01DF91CF916D
:1007D000FF90EF90DF90CF90BDCF80E092E0DF916F
:1007E000CF91FF90EF90DF90CF90089580E003DFEE
:1007F0008A3531F48FEFFFDE8A3511F480E8FBDEB5
:100800008FEF0895882F8F770895672B682B61F4F9
:1008100060E070E080E0F6DF21E030E0882311F056
:1008200020E030E0C90102C080E090E081700895CE
:1008300000C00091780005FD42C0F092A00608E1DA
:100840000093B7060FEF0A950023E9F70091A80679
:1008500007FFECC0E0E0F0E0079116910F3F19F4BC
:100860001F3F09F4E3C02BC03091CF0137FDFCCF0F
:100870003BB72BBFF8012091CA0113E21093CA01C4
:100880000A01E8952093CA013BBF08953BB72BBFEF
:10089000F8012091CA014093CA013DE93093340028
:1008A000E8952093CA013BBF089501E70DBF00E220
:1008B0000EBFC2E9DAE20F94B8000F947C0AF092FE
:1008C000B70600910020109101200A3A154511F059
:1008D0000C940000F0920020F092012000E20093BE
:1008E0007800F6CFFF84EE84DD84CC84BB84AA84B8
:1008F000998488847F806E805D804C80BB81AA81D2
:1009000099818881F0E0EC0FFD1FEF010895FA92C4
:10091000EA92DA92CA92BA92AA929A928A927A92B7
:100920006A925A924A92BA93AA939A938A93089592
:10093000AF93BF93D80101900D9241505040D9F729
:10094000BF91AF9108954091CA01E22FF32F009318
:10095000CA0104914093CA01089540E04BBFF801D9
:1009600058ED54BF208308954A951AF016950795BF
:10097000FBCF08954A951AF0000F111FFBCF089581
:1009800020E008D0E9F708953BBF27913BB702D09C
:10099000D9F708952D9301501040202F212B089551
:1009A00002E1402E05E1502E02E0602EF201362DCC
:1009B0006BBE07911691F201EE5FFF4F3F4F3BBFB9
:1009C000A791B691F201362DEC5FFF4F3F4F3BBF31
:1009D000479157916691242F252B262B21F0FA0160
:1009E000362FD2DF01C0CCDF07E0400E00E0501E02
:1009F000601EA201662D403255416240B8F2089552
:100A0000BD01D801F90104C021912D9341505040FE
:100A1000242F252BC9F7DB010895000000000000FA
:100A2000000000000D947D010D94B2013ECF0FBF78
:100A300008952AE107D00093FA042BE103D0009334
:100A4000FB04089530E002E00F948B000F3F09F49F
:100A50000FE108950F947C0000E00093600000E334
:100A60000F94040A30D10064008301E00093600019
:100A7000AFB7F89451D028E0029FF001EC54F64D46
:100A8000158303950230C0F3D4DF0091C0040093B6
:100A9000C00419D10068008300810061008384EBE9
:100AA00099E20496E6EC80839183E0EC46D10FEF67
:100AB0000583E8EC0081016000830A2FB8DFE3E0E2
:100AC0000D9467008991089500E008950FB7F89498
:100AD00010E41093CA0410E21093CA04E1ECF4E0AD
:100AE000108111601083E9EC108112601083E8EC32
:100AF000108110641083E9EC108111601083E8EC20
:100B000010811068108393CF008308950093C3046D
:100B100008950091C304089500E010E008950AD1FB
:100B2000068F178F20A331A3089566D00091CB04C0
:100B300007FF05C000E814D20F94250429C0F9D19D
:100B4000002331F5EBECC0D004FF18C000E108D25F
:100B50000F94110400E00093C30420E430E010E09F
:100B600062D020E430E010E000E85DD002EE19E24F
:100B70000093BC291093BD2929D10AC0008106FF2A
:100B800002C000E404C0008105FF02C000E2E8D119
:100B90001ED0189531D09ED101FD02C085D1B1F48F
:100BA00002E00093CC040091C5043BD0F801008121
:100BB00005FF06C036D020E2F801269308D106C012
:100BC00000E830D020E2F8012693C0D0E1CFACBFDE
:100BD0009BBF8FBF099119912991399149915991E1
:100BE000699179910990199029903990E991F99139
:100BF00089919991A9910895AA939A938A93FA93C6
:100C0000EA933A922A921A920A927A936A935A93A0
:100C10004A933A932A931A930A938FB79BB7ACB728
:100C2000089500E01AC08A932051304041F02051CD
:100C3000304039F02052304031F080E005C081E092
:100C400003C082E001C083E0EDDF20E0F8012183F2
:100C500026E020838064818335CF68EB79E2202F02
:100C60002F70220F402F440F57DF001F020F43E069
:100C70000F94A200060F171F08959D01E8EC24D0E1
:100C80000F7D008300810F7D00833BD102E005933F
:100C9000A2ECB9E241DF0D930C93539600E2069368
:100CA00000E4069338D1069300E406931D931D9348
:100CB0001C9311961D931D931C9317971D931C93C2
:100CC00010A7D9010895E0ECF4E000810895FFD069
:100CD000002331F0033011F0043009F41FD176D035
:100CE00029D006811781083050E0104009F548E00E
:100CF00022EE39E20AEC19E20F94E800E8ECF4E0A5
:100D00001CD01BD00F94DB05002309F4E6C012D0E1
:100D1000068907FF04C014D002E004A717C0048DA1
:100D2000158D012B09F405C00BD001E004A7EFD00D
:100D30000895DFC0E4EBF9E2089500810062E4CE9B
:100D400000E000A701A702A703A70895BCD00330C5
:100D500011F43BD037C083D080A191A1801B910BAF
:100D6000282F292BA9F47FD0048D158D0217130786
:100D700019F005A5002311F0C7D024C080D081F060
:100D80007BD071F000E0FD0102A703A780A191A133
:100D9000803400E0900720F080E490E005A703C0D5
:100DA00001E00093E129FD0186879787068D178D65
:100DB00022A533A5020F131F008B118B89014AD086
:100DC000A0D0A6D0E4E00D946600A8D056CF7BD08A
:100DD000043011F4FADF3DC0FD018681978162A5E0
:100DE00073A520A131A18B01080F191F201731070E
:100DF00018F4C901861B970BAC0122EE39E2068D6F
:100E0000178D060F171F0F94E80029D023D08034C8
:100E1000904031F42CD0448D558D2417350740F087
:100E200000A311A32CD011F027D059F062D011C02B
:100E300020A131A12017310759F421D011F01CD085
:100E400011F44BD006C00BD00ED000E002A703A7D0
:100E50005ED0B8CF080F191F02A713A70895FD0190
:100E600002A513A5089503D020A731A7089520A5B2
:100E700031A5200F311F089559D00023089545A1B1
:100E800056A167A100E0403050076007089522D0C6
:100E900001FD09C009D039F41AD0013009F449CF55
:100EA000043009F41DD008955ED0E7CF13D001FDC2
:100EB00009C0FADF39F40BD0023009F425C0033041
:100EC00009F40ED008950F947B00A4EBB9E20091D1
:100ED000E02908950091CC04089505E00093E029ED
:100EE000E1ECF9E204E00593E9EBF9E204E00593B3
:100EF000089520DF03E004A700E00687078701D0FC
:100F000007C0E0ECF9E2089504E00093E02903D083
:100F100002E006930895E8EBF9E208950BDF42A1A1
:100F200053A164A1AFDF09F001D00895FA016CBFAD
:100F30001994EBECC9DE02FF08C0F093CA040091DB
:100F4000C02906FF0BC0A3DF09C0008101FF07C055
:100F500002E006D00091B82906FDA8DF16C0B4CD86
:100F60000093CA040895B6DF00FFAECD01E0009300
:100F7000CC04D1DF00E80693C4DF00E8069301E06B
:100F8000EFDFC9DF00E10693A2DE01E00895BD01B5
:100F90004DD12681222371F1A281B3812D913C9103
:100FA000D90114964C91041728F524833583D9016F
:100FB00012964D915C91240F351F06C04C9150E064
:100FC000A40FB51FA483B583A481B581A217B3076D
:100FD00088F411964C911197443081F712964C91F8
:100FE0001297041759F713964C911397141731F76A
:100FF00001E001C000E0DB0108953DD0802F10E04A
:10100000E8D111F400E006C015D0038114812581D8
:10101000D5D101E04DC02FD0802FDBD149F00AD0CF
:10102000008111812281CAD1002311F001E001C0A9
:1010300000E03EC0AEE4B1E2ED91FC91A281B3814B
:1010400002E0809FA00DB11DED91FC9108950D94DB
:10105000120111D00DD139F080E003C0082FCDDF8F
:10106000839509D1D8F300E00093522101E010E00C
:101070000D931C931DC00D947B00A3D1C9F080E09B
:101080000EC0FD0118D044855585668500E04030CE
:101090005007600719F0FA016CBF19958395C6D007
:1010A000A281B381ED91FC9111970481801748F3DF
:1010B000E4E00D9466000281138177D10081F18113
:1010C000E02F08950091CC290F770D946E010091C7
:1010D000CC29002329F00A9541F00A9511F125C089
:1010E00024E030E006E011E21AC025E00EEE10E246
:1010F00040E050E032E0F801E40FF51F6081439FCB
:10110000F001E653FF4D628353834395421798F3F2
:10111000220F2E5F2093CA2030E00AEC10E2A6D006
:1011200005C021E104EF10E2E3CF7CC101E00895A6
:1011300074D0FD014281238104E411E22A9529F053
:101140002A95A1F02A9551F12CC02DD0208130E0B4
:10115000F801008111818AD065D02285338502177C
:10116000130710F40287138701E054C01CD02189B3
:101170004217B8F4F801F9D024E0429F000D111D88
:10118000F80100811181F801228133816FD022E0C2
:10119000FD010085F185E02F2183DECF98DF00235C
:1011A000D9F600E0E2CFF8012081F181E22F089525
:1011B00034D038D0012B59F50F947101002339F147
:1011C000E4E4F1E27BDF2189FD0102812017F8F0E0
:1011D00040DFFD0102810093522120915221222300
:1011E000C1F0E4E4F1E2C1D034E0239F000D111D11
:1011F000045010401BD002831383A0E001C0A395CC
:10120000EAD0A01730F410E04ED00023C1F700E080
:1012100001C001E0A991B9910895BA93AA93AAECEB
:10122000B9E20895FD01068117810895ECE4F1E229
:10123000089521DF93D0068117810130104039F4E1
:1012400017D029F0848117D010F4C1D011F400E038
:101250000CC0FD01A7D02FDFAED00093532121E0B9
:1012600030E017968D0102D001E022CF0D94770176
:10127000ACE4B1E2A8C0FD01B0D080170895AA93F4
:101280008A936CD06ED041F49ED031F0A4818281DB
:101290000A2FB3DE002311F400E002C0182F03D0A0
:1012A0008991A99108950A2FB6CE58D0008107FFE1
:1012B0002DC026813781022F032B09F447C00081FE
:1012C0000F71F1F41181112329F0165069F01250B9
:1012D00061F016C0223000E0304009F0089522E0AD
:1012E00030E00CE411E20AC023CF213000E03040AE
:1012F00009F0089521E030E002E511E2B7DF16CFF2
:10130000013021F501810A3009F593CF0F7101F504
:1013100011811A9581F01250C9F0125019F0145031
:10132000B1F016C01ED091F40AE414E021E0048765
:1013300015872687E4CF15D049F417D00130104027
:1013400029F474DF00810D7F0083D9CF6BC030CFCB
:101350000130E1F701810B30C9F791CFEAECF9E2F6
:10136000089506811781012B089502811381089544
:1013700028D091F08091CE292ED0801768F427D004
:1013800059F054DF0FD0F1DF10D0A081B181FD0101
:1013900012D0102F1DD011F400E003C043DF2085D0
:1013A0000DD086CE0281F3818BCE22E0829F000D8C
:1013B000111DF8010895018512852385F8012CBFC0
:1013C00019940F947B00009152210023089510E09E
:1013D000082FDDDDFACFECE4F1E2E4DF0081F181FA
:1013E000E02F04810895BADF00E0028703870487B5
:1013F000058706870787008B018B008107FF02C0E6
:10140000B0DF81F00091CA29007619F44EDF002385
:1014100041F40091CA290F71013021F4A9DF0023A2
:1014200009F084CE00E0089500E000936F2152D0CF
:101430000F94460A0F94550AD2C00895BA93AA93FE
:10144000AAECB9E20091CA2900760032F9F51091B0
:10145000CB290C9107FF17C0125041F01A9599F54E
:1014600026E030E00EE511E25ED12BC0F8D0408DD1
:10147000518D628D00E040305007600721F1FA0184
:101480006CBF199524C01A9521F01350E1F422D0B5
:1014900018C000916F21002341F000E00F947B0AF7
:1014A0000CE61AE021E01C9609C020E430E002E7D7
:1014B00011E239D101E616E021E01F960D931D934C
:1014C0002C9301E004C0CBD00FE064D000E0A991E0
:1014D000B991089502C000E0089500E0E1D0EAEC7F
:1014E000F9E200E00787008B018B048705870687F8
:1014F0000895F0DF00E0B3D0008F018F028F01E08C
:101500000F947B0AE2E7F1E230812181203001E093
:10151000300709F420C0203003E0300709F43DC053
:101520002130300709F453C0203004E0300739F48B
:101530000F945D0A002300E009F4089550C02330A1
:10154000300721F401E000936F21089523303640E5
:1015500009F452C0C0CF83D0048D158D012309F04A
:101560009CC047815085618540305040604011F4F7
:1015700010D002C027D009F4AECF20E038E0D1D09F
:1015800002EF17E021E0EAECF9E20787108B218BEC
:1015900028C003E002870AE0AACF14D019F023D0B4
:1015A00011F4F7DF98CF048D158D012321F005E3A9
:1015B00017E021E003C00EE617E021E0008F118F55
:1015C000228F0FC004E711E271D000230895FADFE3
:1015D00019F009D011F4DDDF7ECFA7D002C000934F
:1015E000702101E00895E4E5F1E2448155816681CE
:1015F00040305040604008952497E2E7F1E20381D3
:101600001281112319F01A9559F026C00131F0F416
:1016100029D000E024D0008B018B028B038B1CC0EF
:1016200040E0488349834A834B830B8304810A83C8
:1016300016D0088119812A813B81408151816281C4
:101640007381041715072607370728F008D008E02C
:10165000A1DF00E002C0CFD001E024960895E4E5C8
:10166000F1E20895033041F0023031F0043021F00E
:10167000053011F011E001C010E01093712112E06B
:10168000019FF001E955FF4D6081F18104E511E210
:10169000E62F4AE050E00D94800003E001D01BCF1C
:1016A00000935E2102E00093622108950F947A0076
:1016B000A4E5B1E2FD0122893389F801508141801E
:1016C000FD01408A518BF801128103810D901D901C
:1016D0002D903C901397001511052205330540F01D
:1016E00008E000935E210AE00093622100E00BC055
:1016F0000419150B220B330B66D0FD01048B158BDF
:10170000268B378B01E0E5E00D946500A8DF248887
:10171000358964D0222D6CD0A2DF2489358901D08F
:1017200060CF02EB11E20D9477010F947B00A4E5EA
:10173000B1E24ED0012B022B032B49F400E018EF4D
:10174000048B158B068B078B80E098E01BC040D084
:10175000402F412B422B432B99F1003048E01407D6
:1017600080E02040304010F4C80101C098E0A8019A
:1017700066897789481B590B60407040448B558BB4
:10178000668B778B392F2AD0282F32D042EB51E24B
:1017900004C0FD0158D017D02ED08C010197012B29
:1017A000B1F2FA010191AF010F3F99F305E0009307
:1017B0005E2108EE17E021E0FD01008F118F228FDE
:1017C000E4E00D9466000F5F1F4F2F4F3F4F0895C9
:1017D000FD01048915892689378908954089518931
:1017E00062897389048115812681F8012CBF0895CF
:1017F00002EB11E21994008B118B228B338B08952D
:101800002EDF008941894093B2210093B32122E069
:1018100030E085CF24DF17D064897589402F4F735E
:10182000042E112442EB51E2400D511D078010841B
:101830002184F0012CBE199500E0EAECF9E207875B
:10184000008B018BCECE00891189228933890895BE
:10185000B901B2D0208127FDFDCFECEC20812860BA
:101860002083105F98018B010F94E800ECECF1E00D
:101870000081077F008308950F947B00C801A22F89
:10188000B091CA013AD098D0008107FDFDCF82D037
:101890009093C1018093C001A093C40105E337D0A8
:1018A000B093CA01E4E00D9466000F947900C8017A
:1018B000D9012A010DC08D0134D045E08C010F946F
:1018C0009C004AD08096909600EE400E0FEF501E7E
:1018D000042D052979F0082F0F7129F400E2401634
:1018E00000E0500640F72D918C01C6DF01960FEF06
:1018F000400EEDCFE6E00D9464005ED0008107FD60
:10190000FDCF008101FF02C006E301D008950093DE
:10191000CA0121E00BEC11E00D9495003093CA014F
:1019200008953091CA012091CF0127FDFCCF0BD043
:101930002093C001F80141918F014093C401239588
:101940002032B0F3EBCF23E32093CA0120E02093B1
:10195000C2012093C10108952ED0108117FDFDCF43
:10196000DAD005E321C09A938A93802F9091CA011F
:10197000C4DF46D007FDFDCF0DD00093C10111D0CB
:101980008093C40103950032D0F39093CA018991EA
:101990009991089503E30093CA0100E00093C20106
:1019A00008950093C00108950093CA01B2DF8093A7
:1019B000CA01899108958A93EFECF1E00895FBDF65
:1019C000008107FDFDCFB0D000E3EECF01D0F7CF0F
:1019D0000FEFC9CF0F947B00DA01CB01A801622F72
:1019E0000FD007FDFDCF082F092B49F0FA016BBF7F
:1019F00006910D934F5F5F4F6F4F0197F4CF52CF1A
:101A00000091CF0108950F946F0022974A015B0166
:101A1000280139011170802F952DD901801B910B60
:101A2000A040B040CA8807C0EBDF07FDFDCF45E20C
:101A3000002D0F942E000A2D0B2909F455C0DD242A
:101A4000DFDF07FDFDCFEE24FF24F394CC2071F0FF
:101A5000FC01ABBF07911691088319832881312FB0
:101A60002F3F3F4F31F0DD24D39403C00FEF0883A5
:101A700009830A2D0B29C9F0481659066A067B0608
:101A800031F43BD0088334D00A2D0B2971F08C013E
:101A90009D010F5F1F4F2F4F3F4F401651066206AB
:101AA000730619F42AD0098323D0488159818C0107
:101AB0009D010F941C008E5F9F4FAF4FBF4F0FEFE4
:101AC000E00EF01E0E2D0F2909F68C019D0100502D
:101AD000124020403040DD20002E09F0A5CF90DFDD
:101AE00007FDFDCF44E2A4CF2296E1E10D945A0018
:101AF00001E0800E00E0901E08950FEFA00EB01ED2
:101B000005D0601E701EF4010081089501E0400EB2
:101B100000E0501E089510E2019F00E00093C20112
:101B20001092C1010092C0018091CA0108950FBFB7
:101B30000895083049F01FB7F894E0E5F0E02081FF
:101B4000202B2083012F72D008958A938FB7F894A9
:101B50000A9519F00A9559F023C0183019F424D0C9
:101B6000016002C023D00E7F0083E8E616C01ED0BD
:101B7000097F0083183019F417D002600CC01430AC
:101B800011F4008108C01F3F39F400E807870BEB10
:101B9000008B008104600083E0E600810160008327
:101BA000082F44D08991089504E0C3DFE6E5F0E012
:101BB000008108952497E0E7F0E007E01FEF11931C
:101BC0000A95E9F724E001E44AD02CE124D0098306
:101BD0002DE121D0088319810F3F1F4F21F400E42C
:101BE00013E208831983088119810A831B830A8100
:101BF000009362000B810093630034D021E000E485
:101C00002ED00FB7F894E0E5F0E010811E7F10832E
:101C10000DD02496089530E002E00D948B004FB76C
:101C2000F894109504D001230083042F80CFF0E0B6
:101C3000E02FE059FF4FBCCF8A93063011F488E1C2
:101C400001C080E00091510001FB0EF00BD08360D9
:101C5000282F04E404D010E400E0E1DFA3CF10E07B
:101C60000D94950002E065DF0091510001FBE6F75D
:101C70001FEF02E06ACF0A011B01B901A801800130
:101C800091010D94D208E1E0EA930D94EB080A016A
:101C9000A901980180010D9410089A01AB010D94DF
:101CA0003D080A01A90122E730E2200D311D0D9403
:101CB000E8000A01A90128E431E2F7CFE8E4F1E203
:101CC00000919000008300919100018300919200A7
:101CD00002830091930003830895E0EDF1E0008119
:101CE00001FB00E000F90F2708950091CF0107FDE7
:101CF000FCCF40E200E010E020E030E00F942E0046
:101D00000F94CE0801E00895F8940AEA15E5E0E0A2
:101D1000F0E20083118320917900216009E710E04F
:101D20000F949500FFCF089527E402EA10E00F9486
:101D300095000F94C20978940F940F040F944E01EC
:101D4000FFCFDA084821000000D6007220201502DB
:101D500004000000000200230A012B0A0100080011
:101D6000002F0A01350A0103000000390A010000B2
:101D70000004000000410A01000000000000000013
:101D8000000000000075207F209D209D2089209369
:101D9000209D209D209D209D209D209D209D209D5B
:101DA000209D209D209D20000003000000000000D9
:101DB0000000000000000000000000000000000023
:101DC00000000000000000000000000041544D45EC
:101DD0004C00444655204154584D45474131323816
:101DE0004133550004030904FC05010506010606FC
:101DF0000153060100000000120100020000004033
:101E0000EB03E62F040001020001090212000101A8
:101E100000C0320904000000FF0000000A212C214C
:101E20003E211A214021FFFFFFFFFFFFFFFFFFFFC1
:101E3000FFFFFFFFFFFFFFFFFFFFFFFFFFFFFFFFB2
:101E4000FFFFFFFFFFFFFFFFFFFFFFFFFFFFFFFFA2
:101E5000FFFFFFFFFFFFFFFFFFFFFFFFFFFFFFFF92
:101E6000FFFFFFFFFFFFFFFFFFFFFFFFFFFFFFFF82
:1026300093C0000088C0000096C000002FEF0895EE
:1026400077C0000020E108952FEF08952FEF08953F
:102650002FEF08952FEF08952FEF08952FEF08958E
:102660002FEF08952FEF08952FEF08952FEF08957E
:10267000000000000000000000000000000000005A
:10268000000000000000000000000000000000004A
:10269000000000000000000000000000000000003A
:1026A000000000000000000000000000000000002A
:1026B0004154786D65676131323841335520646922
:1026C000736B202870726F746F7479706529003293
:1026D0003031343034323054313234355A53420090
:1026E0006279205374657068616E2042616572770B
:1026F0006F6C6620286D617472697873746F726D87
:1027000040676D782E6465292C20496C6D656E617B
:10271000752032303134000000000000000000005D
:1027200000000000000000000000000000000000A9
:102730002FEF7D3F39F46F3F29F45F3F19F44038A4
:1027400009F4222708952F932227F2DF2F3F11F457
:102750002F9109C0DF9008952F932227E9DF2F3FA3
:10276000F9F32F9100C0B0923B00F601B22E06D0D3
:102770002DE9B092CA0120933400E8952091CF0151
:10278000207CE1F708950000000000000000000038
:102790000000000000000000000000000000000039
:1027A0000000000000000000000000000000000029
:1027B0000000000000000000000000000000000019
:1027C0000000000000000000000000000000000009
:1027D00000000000000000000000000000000000F9
:1027E00000000000000000000000000000000000E9
:1027F00000000000000000000000000000000000D9
:1028000000000000000000000000000000000000C8
:1028100000000000000000000000000000000000B8
:1028200000000000000000000000000000000000A8
:10283000CF93DF93CDB7DEB7C450D440CDBFDEBF5A
:10284000F8948091A00680648093A0068091A406ED
:1028500080648093A4060E9419016F3375468E46EA
:10286000904E61F08091A70680648093A7068BE765
:1028700092E90197F1F700C00000F4CFBE016F5F4D
:102880007B4FCE018D5F9B4F0E940B01CF5FDB4FD3
:1028900088819981C150D440892B69F0CD5FDB4F8D
:1028A00088819981C350D4400196CD5FDB4F8883E6
:1028B0009983C350D44000E010E051C06801E12C7E
:1028C000F12CB701A6015F5F6F4F7F4FCE018F5F85
:1028D0009D4F0E94CA02B701A601CE0101960E9437
:1028E0007801BE016F5F7F4FCE018F5F9D4F0E94C9
:1028F000DD01892B91F117C06801E12CF12CB701A2
:10290000A601CE018F5F9D4F0E947801B701A601FD
:102910005F5F6F4F7F4FCE018F5F9D4F0E94AA0375
:102920000F5F1F4F02C000E010E0CD5FDB4F8881DA
:102930009981C350D44008171907F0F28091A70677
:1029400080648093A7069FE72DE88BE59150204097
:102950008040E1F700C00000F1CF0F5F1F4FCD5F57
:10296000DB4F88819981C350D4400817190708F4B8
:10297000A5CF8091A70680648093A7069FE728E3F0
:1029800081E0915020408040E1F700C00000F1CF8D
:04299000F894FFCFE9
:00000001FF
